:10000000B201B228A400B3172730A3001030142087
:100010000330A300E8301420A30164301420A301AE
:100020000A30142024081F28A2002508A100240853
:10003000A00091202008031DB313B31B0800303E1D
:10004000A7008811081108118316881108110811DA
:100050000F30880583122708B2184C283A30A100C7
:1000600098307D203330A60060201330A100883006
:100070007D20602064307C20602064307C20223031
:10008000A600602028304B200C304B2006304B203F
:10009000B21427084C283214A600321C5A28081122
:1000A000033C031C5F285F200730A100D0307D2077
:1000B000031408003214FE3C0319AD280815321C45
:1000C000321088150F3088052608F0398804881109
:1000D000A60E3218602832307C2003140800A301D9
:1000E000A200FF30A207031CA307031CAD280330A6
:1000F000A100DF307D207128A101E83EA000A10908
:10010000FC30031C8628A00703188328A00764007E
:10011000A10F832820188C28A01C9028000090286C
:100120000800A501A4011030A600210DA40DA50D05
:100130002208A4022308031C230FA5020318A728E2
:100140002208A40723080318230FA5070310A00DF6
:10015000A10DA60B95282008AD2883130313831245
:100160006400080083160E30860087018801811321
:100170008312B801B9010130A300F4308A01702064
:10018000FE308A01202001308A0120202A308A0195
:1001900020202A308A01202041308A012020593035
:1001A0008A0120204B308A01202055308A012020EE
:1001B00054308A01202020308A01202059308A01C1
:1001C000202049308A0120204C308A0120204D30E7
:1001D0008A01202041308A0120205A308A012020C3
:1001E0002A308A0120202A308A012020FE308A010C
:1001F0002020C1308A01202045308A0120204E3045
:100200008A01202044308A0120202E308A012020BB
:1002100045308A0120204C308A01202045308A0157
:1002200020204B308A01202054308A012020523077
:100230008A0120204F308A0120204E308A01202060
:1002400049308A0120204B308A0120201330A3003E
:1002500088308A017020FE308A01202001308A0116
:10026000202048308A01202041308A01202044305B
:100270008A01202049308A01202020308A01202054
:1002800042308A01202041308A01202053308A01E7
:1002900020204C308A01202041308A012020593012
:1002A0008A01202041308A0120204C308A01202000
:1002B00049308A0120204D308A012020FE308A01F9
:1002C0002020C2308A0120204B308A0120204F306C
:1002D0008A0120204C308A01202041308A012020D0
:1002E00059308A01202020308A01202047308A019D
:1002F000202045308A0120204C308A0120205330B4
:100300008A01202049308A0120204E308A01202095
:100310000B30A300B8308A017020FE308A01202003
:1003200001308A0120208701FE3086000612640019
:100330008A110A128618AB290130B800B9018A1156
:100340000A127A220630870064008A110A1286187F
:10035000AB298A01A42964008A110A120619BF294F
:100360000230B800B9018A110A127A225B30870084
:1003700064008A110A120619BF298A01B82964008B
:100380008A110A128619D3290330B800B9018A11DB
:100390000A127A224F30870064008A110A128619E5
:1003A000D3298A01CC2906168316061283128612D7
:1003B00064008A110A128618EC290430B800B901C9
:1003C0008A110A127A226630870064008A110A12A2
:1003D0008618EC298A01E529861264008A110A121E
:1003E0000619012A0530B800B9018A110A127A22C9
:1003F0006D30870064008A110A120619012A8A01E9
:10040000FA29861264008A110A128619162A063001
:10041000B800B9018A110A127A227D30870064007F
:100420008A110A128619162A8A010F2A861683163D
:1004300086128312061364008A110A1286182F2A64
:100440000730B800B9018A110A127A2207308700F2
:1004500064008A110A1286182F2A8A01282A061394
:1004600064008A110A120619442A0830B800B9013A
:100470008A110A127A227F30870064008A110A12D8
:100480000619442A8A013D2A061364008A110A12B9
:100490008619592A0930B800B9018A110A127A223C
:1004A0006F30870064008A110A128619592A8A015E
:1004B000522A0617831606138312861364008A11C4
:1004C0000A120619712AB801B9018A110A127A2290
:1004D0003F30870064008A110A120619712A8A01C6
:1004E0006A2A861783168613643083128A016F2066
:1004F0008A019429FE308A01202081308A0120203F
:1005000042308A01202041308A01202053308A0164
:10051000202049308A0120204C308A01202041309F
:100520008A0120204E308A01202020308A0120209C
:1005300054308A01202055308A01202053308A010E
:1005400020203D308A0120203908A50038088A0182
:100550000220FE308A012020C1308A012020443050
:100560008A01202049308A01202053308A0120202E
:1005700050308A0120204C308A01202041308A01ED
:10058000202059308A01202045308A012020203047
:100590008A01202042308A01202041308A01202017
:1005A0004B308A0120203D308A0120203908A500E7
:1005B00038088A01022032308A016F200800630067
:0405C0008A01DF2AA3
:02400E00753FFC
:00000001FF
